:107800000C94283C0C94433C0C94433C0C94433C17
:107810000C94433C0C94433C0C94433C0C94433CEC
:107820000C94433C0C94433C0C94433C0C94433CDC
:107830000C94433C0C94433C0C94433C0C94433CCC
:107840000C94433C0C94433C0C94433C0C94433CBC
:1078500011241FBECFE5D8E0DEBFCDBF10E0A0E60B
:10786000B0E0E6EEFEE702C005900D92A036B1074B
:10787000D9F711E0A0E6B0E001C01D92A43AB1072B
:10788000E1F70C94363F0C94003C0F92AF93BF93FA
:10789000CF93DF93EF93FF93FC01EA01DB01C895DF
:1078A000099231961197D9F7FF91EF91DF91CF911E
:1078B000BF91AF910F9008950F921F920F93AF93C6
:1078C000BF93CF93DF93EF93FF93FC01EA01DB01BA
:1078D0000990199001E043D032961297C9F7FC0144
:1078E00003E03DD005E03BD0FF91EF91DF91CF91D8
:1078F000BF91AF910F911F900F9008950F931F9319
:10790000EF93FF93FC0103E02AD000E810E0E00FC2
:10791000F11FE617F707B9F7FF91EF911F910F914C
:1079200008950F930F9222D0082E09E018D00F90DF
:107930000F9108950F930F92EF93FF9317D0FC01CF
:1079400060935700C895802DFF91EF910F900F9194
:1079500008950F930BD001E102D00F910895E199A2
:10796000FECF00935700E895FFFF000000915700FD
:1079700000FDFCCF089583E089B98AB188618AB996
:1079800008958AB1877E8AB908958CB95E9BFECF2F
:107990005E9A08958CB1992708958BB199278078C4
:1079A00090700895EF92FF920F931F93CF93DF9300
:1079B0007B01C0E0D0E0C617D70770F48C010E94AD
:1079C000CD3C8823E1F30E94CA3CF80181938F01EA
:1079D0002196CE15DF0598F381E090E0DF91CF91FD
:1079E0001F910F91FF90EF900895EF92FF920F93E8
:1079F0001F93CF93DF937C018B01C0E0D0E0C017D1
:107A0000D10738F4F70181917F010E94C53C21968E
:107A1000F6CF81E090E0DF91CF911F910F91FF9021
:107A2000EF90089540E050E04817590750F42AE6D7
:107A300033E000002150304037FFFBCF4F5F5F4FF6
:107A4000F3CF08950E94C13C0E94000008950E9457
:107A5000CD3C8823E1F30E94CA3C803219F481E0D6
:107A600090E0089585E10E94C53C80E090E0089593
:107A700090E0282F33272138310589F0223831054D
:107A800024F42038310549F00DC02238310549F081
:107A90002839310539F493E005C092E003C091E044
:107AA00001C092E1892F9927089540E050E060914C
:107AB000A0007091A10046175707D0F42091A201B1
:107AC0003091A301E2EAF0E03FBB2EBB2F5F3F4FB6
:107AD00080818DBBE29AE19AE199FECF4F5F5F4FC3
:107AE00031964617570780F33093A3012093A201E4
:107AF000089540E050E06091A0007091A100461709
:107B00005707B0F42091A2013091A301E2EAF0E01E
:107B10003FBB2EBB2F5F3F4FE09A8DB381934F5FEA
:107B20005F4F46175707A0F33093A3012093A2019C
:107B30000895CF93DF93C0E0D0E08091A0009091B2
:107B4000A100C817D907A0F4CE018E559F4F2091F0
:107B5000A2013091A301220F331FAC0160E870E055
:107B6000C9018C0F9D1F0E945C3CC058DF4FE5CFC0
:107B70000E94A93CDF91CF9108958091A20190913C
:107B8000A30142EA50E06091A0007091A100880F2B
:107B9000991F0E94453C0895CF93C0E069E081E0C1
:107BA00090E00E949A3C992784FF03C08F7E0E9438
:107BB000913C0E94CD3C8823E1F30E94CA3C992766
:107BC000823591051CF5803591050CF05CC081343F
:107BD000910509F462C0823491057CF481339105EA
:107BE000B1F18233910524F4C09709F44CC038C137
:107BF0008034910509F438C133C18234910509F408
:107C00005FC08534910509F45EC02AC186359105AF
:107C100009F4F1C0873591054CF48235910509F4DA
:107C20005FC08535910509F469C01AC18437910593
:107C300009F4A4C0853791052CF48436910509F424
:107C400076C00EC18537910509F4C5C009C10E94EF
:107C5000273D882309F4ADCF84E10E94C53C81E42F
:107C60000E94C53C86E50E94C53C82E50E94C53C59
:107C700080E20E94C53C83E50E94C53C84E50E94E9
:107C8000C53C8BE406C00E94273D882309F491CFB0
:107C900084E10E94C53C80E1E4C061E070E080E6E0
:107CA00090E00E94D23C0E94273D882309F481CFB6
:107CB00084E10E94C53C809160000E94383DE9CF7C
:107CC00064E170E008C061E070E080E690E00E944E
:107CD000D23C64E070E080E690E00E94D23CD3CFDA
:107CE0000E94273D882309F464CF60E070E480E0BF
:107CF00090E00E947E3C0E94A93CCACF62E070E006
:107D000080E690E00E94D23C0E94273D882309F43F
:107D100050CF20916000809161009927982F88278B
:107D2000820F911D9093A3018093A201B1CF63E0D4
:107D300070E080E690E00E94D23C2091610080914A
:107D400060009927982F8827820F911D9093A1009A
:107D50008093A000BC0182EA90E00E94D23C0E9485
:107D6000273D882309F425CF80916200863419F4D9
:107D70000E94993D8DCF0E94553D8ACF63E070E00F
:107D800080E690E00E94D23C2091610080916000EA
:107D90009927982F8827820F911D9093A100809397
:107DA000A0000E94273D882309F403CF8091620040
:107DB000863419F40E94BD3D02C00E94793D84E1E1
:107DC0000E94C53C6091A0007091A10082EA90E001
:107DD0000E94F53C60CF0E94273D882309F4E9CE3C
:107DE00084E10E94C53C8EE10E94C53C85E90E9469
:107DF000C53C81E04ECF64E070E080E690E00E94F8
:107E0000D23C0E94273D882309F4D3CE84E10E940E
:107E1000C53C80916000803531F4809161008823F9
:107E200061F4C82F17C0883531F480916100883023
:107E300061F4C3E00FC0803531F480916100883077
:107E400049F4C2E007C0883529F480916100882395
:107E500009F4C1E069E08C2F99270E949A3C19CF60
:107E600085E10E94C53CA5CECF910895CFE5D8E02D
:107E7000DEBFCDBFCEE1F894AEEFB3E00E946A3F23
:107E8000802D843B71F4AFEFB3E00E946A3F802DF8
:107E9000833C39F4ADEFB3E00E946A3F802D99270F
:107EA00081BF0E94BB3C0E94CA3C84E690E00E94D5
:107EB000123D0E94CD3C882319F00E94CC3D04C0A5
:107EC000C150C8BBCC2389F70E94223D80E090E0DE
:107ED0000C94723FE199FECFBFBBAEBBE09A119606
:067EE0000DB20895FFCF72
:040000030000780081
:00000001FF
